:10000000831682309F008601870188018312803029
:100010009F0090309F0098309F000330A500250876
:1000200023208700250828209F002D201F151F1939
:1000300017281E08860083161E0883128800422097
:10004000A50B0F280D288207000008340434013462
:10005000820700009934913481342030A0000000E0
:10006000A00B30280800A530A00000000000A00B65
:10007000372808006330A100000000003320A10BE6
:100080003E2808006330A2006230A3000330A400C1
:1000900000003A20A20B49283320A30B4C28A40BC4
:0400A0004F280800DD
:00000001FF
